:020000040000FA
:0408000063EF09F0A9
:1008100003B283EF05F0F2B4A1EF05F09EB0A9EFAB
:1008200005F09EB2B1EF05F0F2A81AEF04F0F2B2B3
:1008300032EF04F09EB61FEF04F012EF09F09E961F
:1008400000011350000A06E000011350010A06E0FF
:1008500012EF09F02DEC20F012EF09F021EC22F05C
:1008600012EF09F0CD90F2929EA03CEF04F001014E
:10087000533F3CEF04F0542BAEC1B2F1AFC1B3F122
:10088000B0C1B4F1B1C1B5F1AAC1AEF1ABC1AFF124
:10089000ACC1B0F1ADC1B1F1A6C1AAF1A7C1ABF134
:1008A000A8C1ACF1A9C1ADF1A2C1A6F1A3C1A7F144
:1008B000A4C1A8F1A5C1A9F19EC1A2F19FC1A3F154
:1008C000A0C1A4F1A1C1A5F19AC19EF19BC19FF164
:1008D0009CC1A0F19DC1A1F196C19AF197C19BF174
:1008E00098C19CF199C19DF1CECF96F1CFCF97F1F0
:1008F00053C198F154C199F1CF6ACE6A0101536B8B
:10090000546B9E90CD800FBC0F8E0FBA8BEF04F00E
:100910000F8A12EF09F00F8C0FBEC7EF04F096C1DB
:100920009AF197C19BF198C19CF199C19DF19AC12F
:100930009EF19BC19FF19CC1A0F19DC1A1F19EC1FF
:10094000A2F19FC1A3F1A0C1A4F1A1C1A5F1A2C1CF
:10095000A6F1A3C1A7F1A4C1A8F1A5C1A9F1A6C19F
:10096000AAF1A7C1ABF1A8C1ACF1A9C1ADF1AAC16F
:10097000AEF1ABC1AFF1ACC1B0F1ADC1B1F1AEC13F
:10098000B2F1AFC1B3F1B0C1B4F1B1C1B5F1010180
:100990005E6B5F6B606B616B96515E2797515F2357
:1009A00098516023995161239A515E279B515F238F
:1009B0009C5160239D5161239E515E279F515F236F
:1009C000A0516023A1516123A2515E27A3515F234F
:1009D000A4516023A5516123A6515E27A7515F232F
:1009E000A8516023A9516123AA515E27AB515F230F
:1009F000AC516023AD516123AE515E27AF515F23EF
:100A0000B0516023B1516123B2515E27B3515F23CE
:100A1000B4516023B5516123D89001016133603333
:100A20005F335E33D8900101613360335F335E33EF
:100A3000D8900101613360335F335E3300C10CF144
:100A400001C10DF102C10EF103C10FF104C110F19A
:100A500005C111F106C112F107C113F108C114F16A
:100A600009C115F10AC116F10BC117F134C135F1F5
:100A700011B846EF05F00101620E046F010E056F1B
:100A8000000E066F000E076F4FEF05F00101A70E75
:100A9000046F020E056F000E066F000E076F5EC139
:100AA00000F15FC101F160C102F161C103F1C4EC69
:100AB0001EF003BF04D018BE02D018A0108C11A0E5
:100AC00067EF05F010BA67EF05F00F80108A0CC1D0
:100AD00000F10DC101F10EC102F10FC103F110C10E
:100AE00004F111C105F112C106F113C107F114C1DE
:100AF00008F115C109F116C10AF117C10BF135C191
:100B000034F112EF09F00392ABB2AB98AB8803015A
:100B100003EE00F080517F0BE92604C0EFFF802B2D
:100B20008151805D700BD8A48B8200008051815D63
:100B3000700BD8A48B9281518019D8B4079012EF12
:100B400009F0F2940101453F12EF09F0462B12EF34
:100B500009F09E900101533F12EF09F0542B12EF60
:100B600009F09E9211B820EF07F08BB4BFEF05F0AB
:100B700010ACBFEF05F08B84109CC0EF05F08B9498
:100B8000C3CF55F1C4CF56F1C28207B42AEF06F0A5
:100B900047C14BF148C14CF149C14DF14AC14EF139
:100BA0005EC162F15FC163F160C164F161C165F171
:100BB00096C1B6F197C1B7F198C1B8F199C1B9F131
:100BC0009AC1BAF19BC1BBF19CC1BCF19DC1BDF101
:100BD0009EC1BEF19FC1BFF1A0C1C0F1A1C1C1F1D1
:100BE000A2C1C2F1A3C1C3F1A4C1C4F1A5C1C5F1A1
:100BF000A6C1C6F1A7C1C7F1A8C1C8F1A9C1C9F171
:100C0000AAC1CAF1ABC1CBF1ACC1CCF1ADC1CDF140
:100C1000AEC1CEF1AFC1CFF1B0C1D0F1B1C1D1F110
:100C2000B2C1D2F1B3C1D3F1B4C1D4F1B5C1D5F1E0
:100C3000010155515B2756515C23E86A5D230E2E56
:100C40002AEF06F05CC157F15DC158F15B6B5C6B3C
:100C50005D6B078E0201002F12EF09F03C0E006F52
:100C60001950E00BE00AE866128817BE02D017B4EC
:100C7000108E00C10CF101C10DF102C10EF103C1D2
:100C80000FF104C110F105C111F106C112F107C144
:100C900013F108C114F109C115F10AC116F10BC114
:100CA00017F134C135F101018A675EEF06F08B67F9
:100CB0005EEF06F08C675EEF06F08D6762EF06F080
:100CC00092EF06F08EC100F18FC101F190C102F1E7
:100CD00091C103F10101010E046F000E056F000EBA
:100CE000066F000E076FC4EC1EF000C18EF101C14B
:100CF0008FF102C190F103C191F1006787EF06F017
:100D0000016787EF06F0026787EF06F0036792EF4F
:100D100006F08AC18EF18BC18FF18CC190F18DC12B
:100D200091F10F80D57ED5BE6DD0D6CF47F1D7CF0C
:100D300048F145C149F1E86AE8CF4AF118BE02D04E
:100D400018A0108C109047C100F148C101F149C1B1
:100D500002F14AC103F101010A0E046F000E056F92
:100D6000000E066F000E076FC4EC1EF003AF10807C
:100D7000010154A7C8EF06F00F9A0F9C0F9E0101C6
:100D8000000E5E6F600E5F6F3D0E606F080E616F4C
:100D9000010147BFD8EF06F04867D8EF06F0496772
:100DA000D8EF06F04A67D8EF06F0F288FDEF06F0BC
:100DB000F2985E6B5F6B606B616B966B976B986B79
:100DC000996B9A6B9B6B9C6B9D6B9E6B9F6BA06BE7
:100DD000A16BA26BA36BA46BA56BA66BA76BA86B97
:100DE000A96BAA6BAB6BAC6BAD6BAE6BAF6BB06B47
:100DF000B16BB26BB36BB46BB56BD76AD66A0101DA
:100E0000456B466B0CC100F10DC101F10EC102F141
:100E10000FC103F110C104F111C105F112C106F1B6
:100E200013C107F114C108F115C109F116C10AF186
:100E300017C10BF135C134F112EF09F012EF09F0CF
:100E40000201002F79EF08F0D59ED6CF47F1D7CF1A
:100E500048F145C149F1E86AE8CF4AF1D76AD66A54
:100E60000101456B466BD58E1950E00BE00AE86630
:100E7000128817BE02D017B4108E16AE1B8C00C19C
:100E80000CF101C10DF102C10EF103C10FF104C15A
:100E900010F105C111F106C112F107C113F108C12A
:100EA00014F109C115F10AC116F10BC117F134C1D2
:100EB00035F10FA0109A11B869EF07F00101620E29
:100EC000046F010E056F000E066F000E076F72EFC4
:100ED00007F00101A70E046F020E056F000E066FEA
:100EE000000E076F47C100F148C101F149C102F18D
:100EF0004AC103F1C4EC1EF003BF85EF07F018BE32
:100F000002D018A0108C11B00F800CC100F10DC1DF
:100F100001F10EC102F10FC103F110C104F111C1C1
:100F200005F112C106F113C107F114C108F115C191
:100F300009F116C10AF117C10BF135C134F10201F3
:100F40003C0E006F00C10CF101C10DF102C10EF1A8
:100F500003C10FF104C110F105C111F106C112F175
:100F600007C113F108C114F109C115F10AC116F145
:100F70000BC117F134C135F101018A67C7EF07F0E2
:100F80008B67C7EF07F08C67C7EF07F08D67CBEF74
:100F900007F0FBEF07F08EC100F18FC101F190C1A6
:100FA00002F191C103F10101010E046F000E056F02
:100FB000000E066F000E076FC4EC1EF000C18EF12C
:100FC00001C18FF102C190F103C191F10067F0EF0F
:100FD00007F00167F0EF07F00267F0EF07F0036733
:100FE000FBEF07F08AC18EF18BC18FF18CC190F1BC
:100FF0008DC191F10F80109047C100F148C101F1FE
:1010000049C102F14AC103F101010A0E046F000E49
:10101000056F000E066F000E076FC4EC1EF003AFE5
:101020001080010154A721EF08F00F9A0F9C0F9E2A
:101030000101000E5E6F600E5F6F3D0E606F080E67
:10104000616F47C100F148C101F149C102F14AC1D4
:1010500003F10101140E046F050E056F000E066FFB
:10106000000E076FC4EC1EF003AF3AEF08F0F288F1
:101070005FEF08F0F2985E6B5F6B606B616B966B75
:10108000976B986B996B9A6B9B6B9C6B9D6B9E6B34
:101090009F6BA06BA16BA26BA36BA46BA56BA66BE4
:1010A000A76BA86BA96BAA6BAB6BAC6BAD6BAE6B94
:1010B000AF6BB06BB16BB26BB36BB46BB56B0CC198
:1010C00000F10DC101F10EC102F10FC103F110C118
:1010D00004F111C105F112C106F113C107F114C1E8
:1010E00008F115C109F116C10AF117C10BF135C19B
:1010F00034F1E0EC22F01C661ED01BAE11D01B9E1A
:101100001C8E17AE07D0136A040E146E156A2DECF0
:1011100020F011D0136A146A156A2DEC20F00BD060
:101120001BAC09D01B9C1C8C010E136E146A156A33
:1011300021EC22F000D08BB4A5EF08F010ACA5EFA5
:1011400008F08B84109CA6EF08F08B94C3CF55F168
:10115000C4CF56F1C28207B410EF09F047C14BF17A
:1011600048C14CF149C14DF14AC14EF15EC162F135
:101170005FC163F160C164F161C165F196C1B6F10F
:1011800097C1B7F198C1B8F199C1B9F19AC1BAF153
:101190009BC1BBF19CC1BCF19DC1BDF19EC1BEF123
:1011A0009FC1BFF1A0C1C0F1A1C1C1F1A2C1C2F1F3
:1011B000A3C1C3F1A4C1C4F1A5C1C5F1A6C1C6F1C3
:1011C000A7C1C7F1A8C1C8F1A9C1C9F1AAC1CAF193
:1011D000ABC1CBF1ACC1CCF1ADC1CDF1AEC1CEF163
:1011E000AFC1CFF1B0C1D0F1B1C1D1F1B2C1D2F133
:1011F000B3C1D3F1B4C1D4F1B5C1D5F10101555199
:101200005B2756515C23E86A5D230E2E10EF09F030
:101210005CC157F15DC158F15B6B5C6B5D6B078E18
:1012200012EF09F002C0E0FF005001C0D8FF10002B
:10123000A6B218EF09F00CC0A9FF0BC0A8FFA69E2C
:10124000A69CA684F29E550EA76EAA0EA76EA68235
:10125000F28EA694A6B22AEF09F00C2A1200A96E0B
:10126000A69EA69CA680A8500C2A120004012C0E53
:10127000826F39EC0BF0BFEC1FF00C502FEC09F033
:10128000E8CF00F10C502FEC09F0E8CF01F101AFED
:101290004FEF09F00101FF0E026FFF0E036F62ECCA
:1012A0001FF029675BEF09F00401200E826F39EC13
:1012B0000BF060EF09F004012D0E826F39EC0BF09A
:1012C0008CEC1DF01200076A0F6A106A116A126A2C
:1012D0000F010E0EC16E860EC06E030EC26E0F01A0
:1012E000896A110E926E080E8A6EF10E936E8B6AE9
:1012F000980E946EF18EFC0E2FEC09F0E8CF0BF0F7
:101300000BA011800BA211820BA411840BA81188D1
:10131000C90E2FEC09F0E8CF16F0CA0E2FEC09F039
:10132000E8CF17F0CB0E2FEC09F0E8CF18F0CC0E79
:101330002FEC09F0E8CF19F0CD0E2FEC09F0E8CF33
:101340002EF01B6A1C6A0E6A01015B6B5C6B5D6BA5
:10135000576B586BF29A0101476B486B496B4A6BAC
:101360004B6B4C6B4D6B4E6B4F6B506B516B526BB1
:10137000456B466BD76AD66A0F01280ED56EF28A86
:101380009D90B00ECD6E01015E6B5F6B606B616B0B
:10139000626B636B646B656B666B676B686B696BC9
:1013A000536B546BCF6ACE6A0F9A0F9C0F9E9D8031
:1013B000760ECA6E9D8202013C0E006FCC6A160E3C
:1013C0002FEC09F0E8CF00F1170E2FEC09F0E8CF71
:1013D00001F1180E2FEC09F0E8CF02F1190E2FECF5
:1013E00009F0E8CF03F1010103AF11EF0AF0BFEC00
:1013F0001FF0160E0C6E00C10BF018EC09F0170E62
:101400000C6E01C10BF018EC09F0180E0C6E02C145
:101410000BF018EC09F0190E0C6E03C10BF018EC70
:1014200009F000C18AF101C18BF102C18CF103C145
:101430008DF100C18EF101C18FF102C190F103C1A4
:1014400091F11A0E2FEC09F0E8CF00F11B0E2FECF2
:1014500009F0E8CF01F11C0E2FEC09F0E8CF02F102
:101460001D0E2FEC09F0E8CF03F1010103AF67EF88
:101470000AF0BFEC1FF01A0E0C6E00C10BF018EC56
:1014800009F01B0E0C6E01C10BF018EC09F01C0EDC
:101490000C6E02C10BF018EC09F01D0E0C6E03C1AE
:1014A0000BF018EC09F01A0E2FEC09F0E8CF00F160
:1014B0001B0E2FEC09F0E8CF01F11C0E2FEC09F008
:1014C000E8CF02F11D0E2FEC09F0E8CF03F100C1C7
:1014D00092F101C193F102C194F103C195F1240E7F
:1014E000AC6E900EAB6E240EAC6E080EB86E000E95
:1014F000B06E1F0EAF6E0401806B816B0F01900EFA
:10150000AB6E0F019D8A0301806B816BC26B8B9266
:10151000136A146A156A9D8607900001F28EF28C98
:1015200007B035EF1CF00FB0D1EF15F010BED1EFC2
:1015300015F012B8D1EF15F00301805181197F0B1E
:10154000D8B435EF1CF013EE00F081517F0BE1268B
:10155000812BE7CFE8FFE00BD8B435EF1CF023EE8A
:1015600082F0C2513F0BD926E7CFDFFFC22BDF50FD
:10157000780AD8A435EF1CF007808EC100F18FC126
:1015800001F190C102F191C103F10101040E046F58
:10159000000E056F000E066F000E076FC4EC1EF004
:1015A00000AFDCEF0AF00101030E8E6F000E8F6FAB
:1015B000000E906F000E916F03018251720AD8B431
:1015C000B6EF15F08251520AD8B4B6EF15F0825139
:1015D000750AD8B4B6EF15F08251630AD8B4EFEFAC
:1015E00018F08251690AD8B45DEF12F082517A0A7C
:1015F000D8B470EF13F08251490AD8B4FCEF11F05F
:101600008251500AD8B406EF11F08251700AD8B452
:101610004EEF11F08251540AD8B47EEF11F082518E
:10162000740AD8B4C9EF11F08251410AD8B44FEF0F
:101630000CF082514B0AD8B44DEF0BF082516D0A79
:10164000D8B459EF10F082514D0AD8B472EF10F0AF
:101650008251730AD8B4E6EF14F08251530AD8B419
:101660004BEF15F08251590AD8B4AAEF0FF026EFCC
:1016700019F0040114EE00F080517F0BE12682C4C2
:10168000E7FF802B120004010D0E826F39EC0BF086
:101690000A0E826F39EC0BF0120004014B0E826FC0
:1016A00039EC0BF004012C0E826F39EC0BF081B891
:1016B00002D02EB630D003018351430AD8B492EF42
:1016C0000BF003018351630AD8B494EF0BF00301CC
:1016D0008351520AD8B496EF0BF003018351720A7A
:1016E000D8B498EF0BF003018351470AD8B49AEFAE
:1016F0000BF003018351670AD8B49CEF0BF0030190
:101700008351540AD8B49EEF0BF003018351740A3D
:10171000D8B40DEF0CF003018351550AD8B4A0EFF3
:101720000BF082D02E807AD02E9078D02E8276D078
:101730002E9274D02E8472D02E9470D02E866ED0BD
:1017400084C330F185C331F186C332F187C333F1ED
:101750000101296B0DEC20F084EC1FF000C104F1B5
:1017600001C105F102C106F103C107F100EC20F04F
:10177000200EF86EF76AF66A0900F5CF2CF1090021
:10178000F5CF2DF10900F5CF2EF10900F5CF2FF19E
:101790000900F5CF30F10900F5CF31F10900F5CF9F
:1017A00032F10900F5CF33F10101296B0DEC20F086
:1017B00084EC1FF0C4EC1EF00067E6EF0BF001674D
:1017C000E6EF0BF00267E6EF0BF0036701D025D0E0
:1017D00004014E0E826F39EC0BF004016F0E826F24
:1017E00039EC0BF004014D0E826F39EC0BF0040163
:1017F000610E826F39EC0BF00401740E826F39ECCC
:101800000BF00401630E826F39EC0BF00401680EDB
:10181000826F39EC0BF024EF19F02E96CD0E0C6E82
:101820002EC00BF018EC09F0CD0E2FEC09F0E8CF2C
:101830002EF02EB006D00401630E826F39EC0BF04F
:1018400005D00401430E826F39EC0BF02EB206D0A6
:101850000401720E826F39EC0BF005D00401520EB8
:10186000826F39EC0BF02EB406D00401670E826F44
:1018700039EC0BF005D00401470E826F39EC0BF008
:101880002EB606D00401740E826F39EC0BF005D031
:101890000401540E826F39EC0BF024EF19F00401AF
:1018A000410E826F39EC0BF003018351310AD8B439
:1018B000CAEF0EF003018351320AD8B4FAEF0DF0EB
:1018C00003018351330AD8B483EF0DF00301835130
:1018D000340AD8B473EF0CF004013F0E826F39EC78
:1018E0000BF024EF19F0CC0E2FEC09F0E8CF0BF041
:1018F00004012C0E826F39EC0BF003018451310A84
:10190000D8B497EF0CF003018451300AD8B499EFA2
:101910000CF0030184514D0AD8B4A3EF0CF003017D
:101920008451540AD8B4AAEF0CF0C1EF0CF08A84A9
:1019300001D08A940BAE04D00BAC02D00BBA21D0EC
:10194000E00E0B1218D01F0E0B168539E844E00B81
:101950000B1211D0E00E0B1600EC20F085C332F113
:1019600086C333F10101296B0DEC20F084EC1FF0EC
:1019700000511F0B0B12CC0E0C6E0BC00BF018ECB1
:1019800009F00401340E826F39EC0BF004012C0EC7
:10199000826F39EC0BF0CC0E2FEC09F0E8CF19F088
:1019A0008AB406D00401300E826F39EC0BF005D0FA
:1019B0000401310E826F39EC0BF004012C0E826FA2
:1019C00039EC0BF01938E840070BE8CF82F404013A
:1019D000300E822739EC0BF004012C0E826F39ECAB
:1019E0000BF0BFEC1FF019501F0BE8CF00F162ECB9
:1019F0001FF032C182F40401300E822739EC0BF063
:101A000033C182F40401300E822739EC0BF004015B
:101A10002C0E826F39EC0BF0BFEC1FF02CC000F1E4
:101A200000AF0BD0FF0E016FFF0E026FFF0E036FB2
:101A300004012D0E826F39EC0BF062EC1FF031C106
:101A400082F40401300E822739EC0BF032C182F4AB
:101A50000401300E822739EC0BF033C182F404010B
:101A6000300E822739EC0BF004012C0E826F39EC1A
:101A70000BF0BFEC1FF02BC000F162EC1FF031C186
:101A800082F40401300E822739EC0BF032C182F46B
:101A90000401300E822739EC0BF033C182F40401CB
:101AA000300E822739EC0BF004012C0E826F39ECDA
:101AB0000BF0BFEC1FF02DC000F100AF0BD0FF0EFC
:101AC000016FFF0E026FFF0E036F04012D0E826F78
:101AD00039EC0BF062EC1FF031C182F40401300EDE
:101AE000822739EC0BF032C182F40401300E8227D8
:101AF00039EC0BF033C182F40401300E822739EC4B
:101B00000BF024EF19F0CB0E2FEC09F0E8CF0BF01F
:101B100004012C0E826F39EC0BF003018451450A4D
:101B2000D8B4A7EF0DF003018451440AD8B4AAEF4A
:101B30000DF003018451300AD8B4ADEF0DF003016C
:101B40008451310AD8B4B1EF0DF0BCEF0DF00B9E0B
:101B5000B6EF0DF00B8EB6EF0DF0FC0E0B16B6EFD8
:101B60000DF0FC0E0B160B80B6EF0DF0CB0E0C6ECD
:101B70000BC00BF018EC09F00401330E826F39EC46
:101B80000BF004012C0E826F39EC0BF0CB0E2FEC16
:101B900009F0E8CF18F018BED5EF0DF00401450E9E
:101BA000826F39EC0BF0DAEF0DF00401440E826F16
:101BB00039EC0BF004012C0E826F39EC0BF00401B0
:101BC000300E826F39EC0BF004012C0E826F39EC71
:101BD0000BF018B0F3EF0DF00401300E826F39EC0A
:101BE0000BF0F8EF0DF00401310E826F39EC0BF0C1
:101BF00024EF19F0CA0E2FEC09F0E8CF0BF0040126
:101C00002C0E826F39EC0BF003018451450AD8B4D5
:101C100036EF0EF003018451440AD8B439EF0EF0C8
:101C2000030184514D0AD8B442EF0EF003018451F0
:101C3000410AD8B43CEF0EF003018451460AD8B4EF
:101C40003FEF0EF003018451560AD8B44AEF0EF06C
:101C500003018451500AD8B455EF0EF003018451AA
:101C6000520AD8B458EF0EF061EF0EF00B9E5BEF06
:101C70000EF00B8E5BEF0EF00B9C5BEF0EF00B8CFF
:101C80005BEF0EF0FC0E0B1685C3E8FF030B0B1287
:101C90005BEF0EF0C70E0B1685C3E8FF070BE84697
:101CA000E846E8460B125BEF0EF00B845BEF0EF09C
:101CB0000B945BEF0EF0CA0E0C6E0BC00BF018EC21
:101CC00009F0CA0E2FEC09F0E8CF17F00401320E2C
:101CD000826F39EC0BF004012C0E826F39EC0BF0A3
:101CE00017BE7AEF0EF00401450E826F39EC0BF04F
:101CF0007FEF0EF00401440E826F39EC0BF004010B
:101D00002C0E826F39EC0BF017C0E8FF030BE8CF05
:101D100082F40401300E822739EC0BF004012C0E02
:101D2000826F39EC0BF017BC9DEF0EF00401410EF1
:101D3000826F39EC0BF0A2EF0EF00401460E826FB9
:101D400039EC0BF004012C0E826F39EC0BF017C04C
:101D5000E8FF380BE842E842E842E8CF82F40401A9
:101D6000300E822739EC0BF004012C0E826F39EC17
:101D70000BF017B4C3EF0EF00401520E826F39EC72
:101D80000BF0C8EF0EF00401500E826F39EC0BF02F
:101D900024EF19F0C90E2FEC09F0E8CF0BF0040185
:101DA0002C0E826F39EC0BF003018451450AD8B434
:101DB000E8EF0EF003018451440AD8B4EBEF0EF0C3
:101DC000030184514D0AD8B4EEEF0EF0FCEF0EF093
:101DD0000B9EF6EF0EF00B8EF6EF0EF0F80E0B16D4
:101DE00085C3E8FF070B0B12F6EF0EF0C90E0C6E61
:101DF0000BC00BF018EC09F00401310E826F39ECC6
:101E00000BF004012C0E826F39EC0BF0C90E2FEC95
:101E100009F0E8CF16F016BE06D00401450E826F19
:101E200039EC0BF005D00401440E826F39EC0BF055
:101E300004012C0E826F39EC0BF016C0E8FF070B83
:101E4000E8CF82F40401300E822739EC0BF0040154
:101E50002C0E826F39EC0BF00780BFEC1FF027C00F
:101E6000E8FF003B00430043030B62EC1FF033C16B
:101E700082F40401300E822739EC0BF004012C0EA1
:101E8000826F39EC0BF0BFEC1FF027C001F1019F0E
:101E9000019D28C000F1010162EC1FF02FC182F406
:101EA0000401300E822739EC0BF030C182F40401BA
:101EB000300E822739EC0BF031C182F40401300E70
:101EC000822739EC0BF032C182F40401300E8227F4
:101ED00039EC0BF033C182F40401300E822739EC67
:101EE0000BF004012C0E826F39EC0BF0BFEC1FF0ED
:101EF00029C001F12AC000F1D89001330033D890F5
:101F000001330033010162EC1FF02FC182F40401A0
:101F1000300E822739EC0BF030C182F40401300E10
:101F2000822739EC0BF031C182F40401300E822794
:101F300039EC0BF032C182F40401300E822739EC07
:101F40000BF033C182F40401300E822739EC0BF020
:101F500024EF19F0FC0E2FEC09F0E8CF0BF0030191
:101F60008351520AD8B4E1EF0FF003018351720A92
:101F7000D8B4E4EF0FF003018351500AD8B4E7EF6F
:101F80000FF003018351700AD8B4EAEF0FF0030198
:101F90008351550AD8B4EDEF0FF003018351750A50
:101FA000D8B4F0EF0FF003018351430AD8B4F9EF2E
:101FB0000FF003018351630AD8B4FCEF0FF005EF73
:101FC00010F00B90FFEF0FF00B80FFEF0FF00B9274
:101FD000FFEF0FF00B82FFEF0FF00B94FFEF0FF00E
:101FE0000B84FFEF0FF00B96FFEF0FF00B86FFEF68
:101FF0000FF00B98FFEF0FF00B88FFEF0FF0FC0EC8
:102000000C6E0BC00BF018EC09F00401590E826F36
:1020100039EC0BF01190119211941198FC0E2FECE9
:1020200009F0E8CF0BF00BA011800BA211820BA4DA
:1020300011840BA8118811A025EF10F00401520E95
:10204000826F39EC0BF02AEF10F00401720E826FF0
:1020500039EC0BF011A834EF10F00401430E826F3D
:1020600039EC0BF039EF10F00401630E826F39EC9C
:102070000BF011A243EF10F00401500E826F39EC07
:102080000BF048EF10F00401700E826F39EC0BF08A
:1020900011A452EF10F00401550E826F39EC0BF0D1
:1020A00057EF10F00401750E826F39EC0BF024EF3E
:1020B00019F004016D0E826F39EC0BF003018351AE
:1020C000300AD8B4B6EF10F003018351310AD8B406
:1020D000C9EF10F003018351320AD8B4DCEF10F0DD
:1020E00026EF19F081B803D02EB424EF19F00401C3
:1020F0004D0E826F39EC0BF000EC20F084C331F10F
:1021000085C332F186C333F10101296B0DEC20F058
:1021100084EC1FF003018351300AD8B49EEF10F015
:1021200003018351310AD8B4A6EF10F003018351A3
:10213000320AD8B4AEEF10F026EF19F0FD0E0C6E97
:1021400000C10BF018EC09F0B6EF10F0FE0E0C6EAB
:1021500000C10BF018EC09F0C9EF10F0FF0E0C6E87
:1021600000C10BF018EC09F0DCEF10F00401300EA8
:10217000826F39EC0BF004012C0E826F39EC0BF0FE
:10218000BFEC1FF0FD0E2FEC09F0E8CF00F1EDEFF2
:1021900010F00401310E826F39EC0BF004012C0EAB
:1021A000826F39EC0BF0BFEC1FF0FE0E2FEC09F044
:1021B000E8CF00F1EDEF10F00401320E826F39EC40
:1021C0000BF0BFEC1FF004012C0E826F39EC0BF00A
:1021D000FF0E2FEC09F0E8CF00F162EC1FF031C1E7
:1021E00082F40401300E822739EC0BF032C182F404
:1021F0000401300E822739EC0BF033C182F4040164
:10220000300E822739EC0BF024EF19F081B803D09F
:102210002EB2FCEF11F083C32AF184C32BF185C3E6
:102220002CF186C32DF187C32EF188C32FF189C30A
:1022300030F18AC331F18BC332F18CC333F1010128
:102240000DEC20F084EC1FF0160E0C6E00C10BF0AC
:1022500018EC09F0170E0C6E01C10BF018EC09F028
:10226000180E0C6E02C10BF018EC09F0190E0C6E72
:1022700003C10BF018EC09F000C18AF101C18BF128
:1022800002C18CF103C18DF100C18EF101C18FF14A
:1022900002C190F103C191F1FCEF11F081B803D0BC
:1022A0002EB2FCEF11F083C32AF184C32BF185C356
:1022B0002CF186C32DF187C32EF188C32FF189C37A
:1022C00030F18AC331F18BC332F18CC333F1010198
:1022D0000DEC20F084EC1FF000C18AF101C18BF1FC
:1022E00002C18CF103C18DF100C18EF101C18FF1EA
:1022F00002C190F103C191F1FCEF11F081B803D05C
:102300002EB2FCEF11F083C32AF184C32BF185C3F5
:102310002CF186C32DF187C32EF188C32FF189C319
:1023200030F18AC331F18CC332F18DC333F1010135
:102330000DEC20F084EC1FF00101000E046F000E84
:10234000056F010E066F000E076FD5EC1EF01A0E1A
:102350000C6E00C10BF018EC09F01B0E0C6E01C1E5
:102360000BF018EC09F01C0E0C6E02C10BF018EC0F
:1023700009F01D0E0C6E03C10BF018EC09F000C142
:1023800092F101C193F102C194F103C195F1FCEF07
:1023900011F081B803D02EB2FCEF11F083C32AF103
:1023A00084C32BF185C32CF186C32DF187C32EF195
:1023B00088C32FF189C330F18AC331F18CC332F164
:1023C0008DC333F101010DEC20F084EC1FF001010D
:1023D000000E046F000E056F010E066F000E076FF2
:1023E000D5EC1EF000C192F101C193F102C194F14C
:1023F00003C195F1FCEF11F0160E2FEC09F0E8CFB8
:1024000000F1170E2FEC09F0E8CF01F1180E2FECB8
:1024100009F0E8CF02F1190E2FEC09F0E8CF03F133
:1024200062EC1FF045EC1DF00401730E826F39EC75
:102430000BF004012C0E826F39EC0BF08AC100F115
:102440008BC101F18CC102F18DC103F162EC1FF06F
:1024500045EC1DF00401730E826F39EC0BF00401A2
:102460002C0E826F39EC0BF01A0E2FEC09F0E8CF2E
:1024700000F11B0E2FEC09F0E8CF01F11C0E2FEC40
:1024800009F0E8CF02F11D0E2FEC09F0E8CF03F1BF
:1024900041EC19F004012C0E826F39EC0BF092C163
:1024A00000F193C101F194C102F195C103F141EC36
:1024B00019F043EC0BF026EF19F00401690E826F5E
:1024C00039EC0BF004012C0E826F39EC0BF001019A
:1024D000040E006F000E016F000E026F000E036FFE
:1024E00062EC1FF02CC182F40401300E822739EC1B
:1024F0000BF02DC182F40401300E822739EC0BF071
:102500002EC182F40401300E822739EC0BF02FC16A
:1025100082F40401300E822739EC0BF030C182F4D2
:102520000401300E822739EC0BF031C182F4040132
:10253000300E822739EC0BF032C182F40401300EE8
:10254000822739EC0BF033C182F40401300E82276C
:1025500039EC0BF004012C0E826F39EC0BF0010109
:10256000030E006F000E016F000E026F000E036F6E
:1025700062EC1FF02CC182F40401300E822739EC8A
:102580000BF02DC182F40401300E822739EC0BF0E0
:102590002EC182F40401300E822739EC0BF02FC1DA
:1025A00082F40401300E822739EC0BF030C182F442
:1025B0000401300E822739EC0BF031C182F40401A2
:1025C000300E822739EC0BF032C182F40401300E58
:1025D000822739EC0BF033C182F40401300E8227DC
:1025E00039EC0BF004012C0E826F39EC0BF0010179
:1025F0002F0E006F000E016F000E026F000E036FB2
:1026000062EC1FF02CC182F40401300E822739ECF9
:102610000BF02DC182F40401300E822739EC0BF04F
:102620002EC182F40401300E822739EC0BF02FC149
:1026300082F40401300E822739EC0BF030C182F4B1
:102640000401300E822739EC0BF031C182F4040111
:10265000300E822739EC0BF032C182F40401300EC7
:10266000822739EC0BF033C182F40401300E82274B
:1026700039EC0BF004012C0E826F39EC0BF0200EBC
:10268000F86EF76AF66A04010900F5CF82F439ECB6
:102690000BF00900F5CF82F439EC0BF00900F5CF0F
:1026A00082F439EC0BF00900F5CF82F439EC0BF031
:1026B0000900F5CF82F439EC0BF00900F5CF82F474
:1026C00039EC0BF00900F5CF82F439EC0BF009007E
:1026D000F5CF82F439EC0BF043EC0BF026EF19F058
:1026E00081B803D02EB024EF19F08351630AD8A427
:1026F00024EF19F08451610AD8A424EF19F0855110
:102700006C0AD8A424EF19F08651410A42E08651A0
:10271000440A1BE08651420AD8B4DCEF13F086511C
:10272000350AD8B4B0EF1AF08651360AD8B405EF9E
:102730001BF08651370AD8B46EEF1BF08651380A69
:10274000D8B4CCEF1BF024EF19F00798079A0401D6
:102750007A0E826F39EC0BF00401780E826F39EC3F
:102760000BF00401640E826F39EC0BF081A8C0EF0E
:1027700013F00401550E826F39EC0BF0C5EF13F026
:1027800004014C0E826F39EC0BF043EC0BF026EF9A
:1027900019F00788079A04017A0E826F39EC0BF062
:1027A0000401410E826F39EC0BF00401610E826F5F
:1027B00039EC0BF0B6EF13F00798078A04017A0E94
:1027C000826F39EC0BF00401420E826F39EC0BF092
:1027D0000401610E826F39EC0BF0B6EF13F00101CA
:1027E0006667FAEF13F06767FAEF13F06867FAEFBE
:1027F00013F0696715D04F6705EF14F0506705EFC8
:1028000014F0516705EF14F052670AD00101000E71
:10281000006F000E016F000E026F000E036F1200BA
:1028200011B80AD00101620E046F010E056F000E8F
:10283000066F000E076F09D00101A70E046F020E8C
:10284000056F000E066F000E076F66C100F167C1CD
:1028500001F168C102F169C103F1C4EC1EF003BFCC
:10286000A2EF14F0119A119C0101000E046FA80E42
:10287000056F550E066F020E076F66C100F167C146
:1028800001F168C102F169C103F166C186F167C156
:1028900087F168C188F169C189F1C4EC1EF003BFFA
:1028A0000BD00101000E866FA80E876F550E886F42
:1028B000020E896F118A119C0E0E2FEC09F0E8CFE1
:1028C00018F10F0E2FEC09F0E8CF19F1100E2FECD4
:1028D00009F0E8CF1AF1110E2FEC09F0E8CF1BF147
:1028E0000DEC1EF086C104F187C105F188C106F127
:1028F00089C107F1C4EC1EF00782D1EC1DF00DEC8C
:102900001EF00792D1EC1DF086C100F187C101F1E4
:1029100088C102F189C103F10792D1EC1DF0CC0E00
:10292000046FE00E056F870E066F050E076FC4EC8F
:102930001EF000C118F101C119F102C11AF103C161
:102940001BF13BD0119C119A0101800E006F1A0EF1
:10295000016F060E026F000E036F4FC104F150C1EC
:1029600005F151C106F152C107F1C4EC1EF003AFED
:1029700005D0BFEC1FF0118C119A12000E0E2FEC37
:1029800009F0E8CF18F10F0E2FEC09F0E8CF19F19C
:10299000100E2FEC09F0E8CF1AF1110E2FEC09F010
:1029A000E8CF1BF14FC100F150C101F151C102F15B
:1029B00052C103F10782D1EC1DF018C100F119C119
:1029C00001F11AC102F11BC103F112000401730EDF
:1029D000826F39EC0BF004012C0E826F39EC0BF096
:1029E000078462C166F163C167F164C168F165C1C2
:1029F00069F14BC14FF14CC150F14DC151F14EC184
:102A000052F157C159F158C15AF107940CEC15F025
:102A100043EC0BF026EF19F066C100F167C101F13C
:102A200068C102F169C103F1010162EC1FF045ECDC
:102A30001DF00401630E826F39EC0BF004012C0EC3
:102A4000826F39EC0BF04FC100F150C101F151C15F
:102A500002F152C103F1010162EC1FF045EC1DF0DF
:102A60000401660E826F39EC0BF004012C0E826FAC
:102A700039EC0BF0BFEC1FF059C100F15AC101F164
:102A8000010162EC1FF045EC1DF00401740E826F31
:102A900039EC0BF0120010820401530E826F39ECF6
:102AA0000BF004012C0E826F39EC0BF083C32AF17A
:102AB00084C32BF185C32CF186C32DF187C32EF17E
:102AC00088C32FF189C330F18AC331F18BC332F14E
:102AD0008CC333F101010DEC20F084EC1FF000C138
:102AE00066F101C167F102C168F103C169F18EC3EA
:102AF0002AF18FC32BF190C32CF191C32DF192C316
:102B00002EF193C32FF194C330F195C331F196C3E5
:102B100032F197C333F101010DEC20F084EC1FF08A
:102B200000C14FF101C150F102C151F103C152F195
:102B300000EC20F099C32FF19AC330F19BC331F11F
:102B40009CC332F19DC333F101010DEC20F084EC04
:102B50001FF000C159F101C15AF10CEC15F004014C
:102B60002C0E826F39EC0BF0C5EF15F0118E18A00A
:102B700002D018AE108C17BE02D017A4108E82514E
:102B8000520A02E10F8201D00F928251750A02E1CE
:102B9000108401D010948251550A02E1108601D0B0
:102BA000109611A003D011A401D01084078410B294
:102BB00033EF16F010A41FEF16F0B6C166F1B7C1DF
:102BC00067F1B8C168F1B9C169F1BAC16AF1BBC1B5
:102BD0006BF1BCC16CF1BDC16DF1BEC16EF1BFC185
:102BE0006FF1C0C170F1C1C171F1C2C172F1C3C155
:102BF00073F1C4C174F1C5C175F1C6C176F1C7C125
:102C000077F1C8C178F1C9C179F1CAC17AF1CBC1F4
:102C10007BF1CCC17CF1CDC17DF1CEC17EF1CFC1C4
:102C20007FF1D0C180F1D1C181F1D2C182F1D3C194
:102C300083F1D4C184F1D5C185F127EF16F062C1CB
:102C400066F163C167F164C168F165C169F14BC1A7
:102C50004FF14CC150F14DC151F14EC152F157C12C
:102C600059F158C15AF107940FA055EF16F0010120
:102C7000926742EF16F0936742EF16F0946742EFC7
:102C800016F0956746EF16F055EF16F0EFEC13F0DF
:102C900092C104F193C105F194C106F195C107F108
:102CA000C4EC1EF003BFECEF18F0EFEC13F00101E1
:102CB000000E046F000E056F010E066F000E076F09
:102CC000F5EC1EF011A02CD011A22AD062EC1FF05E
:102CD000296701D007D004012D0E826F39EC0BF06B
:102CE000EAEF18F030C182F40401300E822739EC8B
:102CF0000BF031C182F40401300E822739EC0BF065
:102D000032C182F40401300E822739EC0BF033C15A
:102D100082F40401300E822739EC0BF0EAEF18F050
:102D200012A8C5D0129819C01AF01A3A1A42070E02
:102D30001A1600011A50000AD8B423EF17F0000148
:102D40001A50010AD8B4AFEF16F000011A50020A67
:102D5000D8B4ADEF16F055EF17F055EF17F0BFEC04
:102D60001FF029C001F12AC000F1D89001330033CF
:102D7000D890013300330101630E046F000E056F1C
:102D8000000E066F000E076FF5EC1EF0280E046FA4
:102D9000000E056F000E066F000E076FC4EC1EF0EC
:102DA00000C12CF0BFEC1FF027C001F1019F019D75
:102DB00028C000F10101A40E046F000E056F000E83
:102DC000066F000E076FF5EC1EF000C12BF000C17E
:102DD00004F101C105F102C106F103C107F1640E5E
:102DE000006F000E016F000E026F000E036FC4EC47
:102DF0001EF0050E046F000E056F000E066F000E2C
:102E0000076FF5EC1EF000C104F101C105F102C12C
:102E100006F103C107F1BFEC1FF02CC000F1C4ECB8
:102E20001EF000C12DF02DC0E8FF050F2C5C03E75C
:102E30008A8455EF17F02DC0E8FF0A0F2C5C01E6DD
:102E40008A9455EF17F000C124F101C125F102C1A8
:102E500026F103C127F1BFEC1FF0C5EC1FF019509C
:102E60001F0BE8CF00F10101640E046F000E056F27
:102E7000000E066F000E076FD5EC1EF024C104F1A2
:102E800025C105F126C106F127C107F1C4EC1EF0EA
:102E900003BF02D08A9401D08A8424C100F125C1E5
:102EA00001F126C102F127C103F1ECEF18F000C1D6
:102EB00024F101C125F102C126F103C127F110AEB1
:102EC0004CD0109E00C108F101C109F102C10AF104
:102ED00003C10BF162EC1FF030C1D6F131C1D7F163
:102EE00032C1D8F133C1D9F108C100F109C101F1F2
:102EF0000AC102F10BC103F101016C0E046F070E50
:102F0000056F000E066F000E076FC4EC1EF003BFC6
:102F100004D00101550EDA6F1CD008C100F109C1BF
:102F200001F10AC102F10BC103F10101A40E046F0A
:102F3000060E056F000E066F000E076FC4EC1EF044
:102F400003BF04D001017F0EDA6F03D00101FF0E31
:102F5000DA6F1B8E11AEECEF18F024C100F125C121
:102F600001F126C102F127C103F110A4BFEF17F050
:102F70000401750E826F39EC0BF0C4EF17F00401F9
:102F8000720E826F39EC0BF004012C0E826F39EC5B
:102F90000BF062EC1FF02967D3EF17F00401200E4D
:102FA000826FD6EF17F004012D0E826F39EC0BF013
:102FB00030C182F40401300E822739EC0BF031C1AC
:102FC00082F40401300E822739EC0BF004012E0E3E
:102FD000826F39EC0BF032C182F40401300E82278B
:102FE00039EC0BF033C182F40401300E822739EC46
:102FF0000BF004016D0E826F39EC0BF004012C0E06
:10300000826F39EC0BF04FC100F150C101F151C199
:1030100002F152C103F1010162EC1FF045EC1DF019
:103020000401480E826F39EC0BF004017A0E826FB6
:1030300039EC0BF004012C0E826F39EC0BF066C1F9
:1030400000F167C101F168C102F169C103F1010139
:1030500062EC1FF045EC1DF00401630E826F39EC49
:103060000BF004012C0E826F39EC0BF066C100F1FD
:1030700067C101F168C102F169C103F101010A0EE2
:10308000046F000E056F000E066F000E076FD5EC83
:103090001EF0000E046F120E056F000E066F000E7C
:1030A000076FF5EC1EF062EC1FF02AC182F40401F8
:1030B000300E822739EC0BF02BC182F40401300E64
:1030C000822739EC0BF02CC182F40401300E8227E8
:1030D00039EC0BF02DC182F40401300E822739EC5B
:1030E0000BF02EC182F40401300E822739EC0BF074
:1030F0002FC182F40401300E822739EC0BF030C16D
:1031000082F40401300E822739EC0BF004012E0EFC
:10311000826F39EC0BF031C182F40401300E82274A
:1031200039EC0BF032C182F40401300E822739EC05
:103130000BF033C182F40401300E822739EC0BF01E
:103140000401730E826F39EC0BF004012C0E826FB8
:1031500039EC0BF0BFEC1FF059C100F15AC101F17D
:1031600050EC1AF00FB2B8EF18F00FA0EAEF18F019
:1031700004012C0E826F39EC0BF0200EF86EF76A0A
:10318000F66A04010900F5CF82F439EC0BF009006E
:10319000F5CF82F439EC0BF00900F5CF82F439EC6D
:1031A0000BF00900F5CF82F439EC0BF00900F5CFF4
:1031B00082F439EC0BF00900F5CF82F439EC0BF016
:1031C0000900F5CF82F439EC0BF00900F5CF82F459
:1031D00039EC0BF043EC0BF00F9026EF19F00401E3
:1031E000630E826F39EC0BF004012C0E826F39EC08
:1031F0000BF02CEC19F004012C0E826F39EC0BF063
:103200009FEC19F004012C0E826F39EC0BF01BECD3
:103210001AF004012C0E826F39EC0BF00101F80E4C
:10322000006FCD0E016F660E026F030E036F41EC4F
:1032300019F004012C0E826F39EC0BF031EC1AF00E
:1032400043EC0BF026EF19F043EC0BF00301C26BDB
:103250000790109235EF1CF0D8900E0E2FEC09F06D
:10326000E8CF00F10F0E2FEC09F0E8CF01F1100EBE
:103270002FEC09F0E8CF02F1110E2FEC09F0E8CFA6
:1032800003F10101000E046F000E056F010E066FC1
:10329000000E076FF5EC1EF062EC1FF02AC182F4FD
:1032A0000401300E822739EC0BF02BC182F40401AB
:1032B000300E822739EC0BF02CC182F40401300E61
:1032C000822739EC0BF02DC182F40401300E8227E5
:1032D00039EC0BF02EC182F40401300E822739EC58
:1032E0000BF02FC182F40401300E822739EC0BF071
:1032F00030C182F40401300E822739EC0BF031C169
:1033000082F40401300E822739EC0BF004012E0EFA
:10331000826F39EC0BF032C182F40401300E822747
:1033200039EC0BF033C182F40401300E822739EC02
:103330000BF004016D0E826F39EC0BF01200120ECF
:103340002FEC09F0E8CF00F1130E2FEC09F0E8CFD5
:1033500001F1140E2FEC09F0E8CF02F1150E2FEC5D
:1033600009F0E8CF03F101010A0E046F000E056FAA
:10337000000E066F000E076FD5EC1EF0000E046FF6
:10338000120E056F000E066F000E076FF5EC1EF0B3
:1033900062EC1FF02AC182F40401300E822739EC5E
:1033A0000BF02BC182F40401300E822739EC0BF0B4
:1033B0002CC182F40401300E822739EC0BF02DC1B0
:1033C00082F40401300E822739EC0BF02EC182F416
:1033D0000401300E822739EC0BF02FC182F4040176
:1033E000300E822739EC0BF030C182F40401300E2C
:1033F000822739EC0BF004012E0E826F39EC0BF0B2
:1034000031C182F40401300E822739EC0BF032C155
:1034100082F40401300E822739EC0BF033C182F4C0
:103420000401300E822739EC0BF00401730E826F19
:1034300039EC0BF012000A0E2FEC09F0E8CF00F186
:103440000B0E2FEC09F0E8CF01F10C0E2FEC09F078
:10345000E8CF02F10D0E2FEC09F0E8CF03F150EFA9
:103460001AF0060E2FEC09F0E8CF00F1070E2FEC52
:1034700009F0E8CF01F1080E2FEC09F0E8CF02F1D6
:10348000090E2FEC09F0E8CF03F150EF1AF001011B
:10349000BFEC1FF0078457C100F158C101F1079438
:1034A0000101E80E046F800E056F000E066F000E1E
:1034B000076FD5EC1EF0000E046F040E056F000EB2
:1034C000066F000E076FF5EC1EF0880E046F130EEA
:1034D000056F000E066F000E076FC4EC1EF00A0E9B
:1034E000046F000E056F000E066F000E076FF5ECFF
:1034F0001EF062EC1FF00101296784EF1AF004014D
:10350000200E826F87EF1AF004012D0E826F39ECC6
:103510000BF030C182F40401300E822739EC0BF03D
:1035200031C182F40401300E822739EC0BF032C134
:1035300082F40401300E822739EC0BF004012E0EC8
:10354000826F39EC0BF033C182F40401300E822714
:1035500039EC0BF00401430E826F39EC0BF01200D2
:1035600087C32AF188C32BF189C32CF18AC32DF1BB
:103570008BC32EF18CC32FF18DC330F18EC331F18B
:1035800090C332F191C333F10101296B0DEC20F0AE
:1035900084EC1FF00101000E046F000E056F010E98
:1035A000066F000E076FD5EC1EF00E0E0C6E00C1FC
:1035B0000BF018EC09F00F0E0C6E01C10BF018ECBB
:1035C00009F0100E0C6E02C10BF018EC09F0110E90
:1035D0000C6E03C10BF018EC09F004017A0E826F37
:1035E00039EC0BF004012C0E826F39EC0BF0040166
:1035F000350E826F39EC0BF004012C0E826F39EC22
:103600000BF02CEC19F0C5EF13F087C32AF188C337
:103610002BF189C32CF18AC32DF18BC32EF18CC3FE
:103620002FF18DC330F18EC331F190C332F191C3CC
:1036300033F10101296B0DEC20F084EC1FF0880EB2
:10364000046F130E056F000E066F000E076FC9ECB6
:103650001EF0000E046F040E056F000E066F000EC4
:10366000076FD5EC1EF00101E80E046F800E056FA8
:10367000000E066F000E076FF5EC1EF00A0E0C6EC2
:1036800000C10BF018EC09F00B0E0C6E01C10BF031
:1036900018EC09F00C0E0C6E02C10BF018EC09F0DE
:1036A0000D0E0C6E03C10BF018EC09F004017A0E3C
:1036B000826F39EC0BF004012C0E826F39EC0BF0A9
:1036C0000401360E826F39EC0BF004012C0E826F70
:1036D00039EC0BF01BEC1AF0C5EF13F087C32AF19D
:1036E00088C32BF189C32CF18AC32DF18BC32EF132
:1036F0008CC32FF18DC330F18FC331F190C332F100
:1037000091C333F101010DEC20F084EC1FF0000EA9
:10371000046F120E056F000E066F000E076FD5ECDA
:103720001EF001010A0E046F000E056F000E066FF9
:10373000000E076FF5EC1EF0120E0C6E00C10BF0C0
:1037400018EC09F0130E0C6E01C10BF018EC09F027
:10375000140E0C6E02C10BF018EC09F0150E0C6E75
:1037600003C10BF018EC09F004017A0E826F39ECFA
:103770000BF004012C0E826F39EC0BF00401370EB4
:10378000826F39EC0BF004012C0E826F39EC0BF0D8
:103790009FEC19F0C5EF13F087C32AF188C32BF112
:1037A00089C32CF18AC32DF18BC32EF18CC32FF169
:1037B0008DC330F18EC331F190C332F191C333F137
:1037C0000101296B0DEC20F084EC1FF0880E046FD2
:1037D000130E056F000E066F000E076FC9EC1EF08A
:1037E000000E046F040E056F000E066F000E076FCB
:1037F000D5EC1EF00101E80E046F800E056F000E7F
:10380000066F000E076FF5EC1EF0060E0C6E00C181
:103810000BF018EC09F0070E0C6E01C10BF018EC60
:1038200009F0080E0C6E02C10BF018EC09F0090E3D
:103830000C6E03C10BF018EC09F004017A0E826FD4
:1038400039EC0BF004012C0E826F39EC0BF0040103
:10385000380E826F39EC0BF004012C0E826F39ECBC
:103860000BF031EC1AF0C5EF13F081B803D02EB095
:10387000F3EF1CF007A8ADEF1CF00101800E006F04
:103880001A0E016F060E026F000E036F4BC104F19A
:103890004CC105F14DC106F14EC107F1C4EC1EF05B
:1038A00003BFF3EF1CF03FEC1DF04BC100F14CC126
:1038B00001F14DC102F14EC103F10782D1EC1DF0BF
:1038C00018C104F119C105F11AC106F11BC107F1B4
:1038D000F80E006FCD0E016F660E026F030E036FC0
:1038E000C4EC1EF00E0E0C6E00C10BF018EC09F0CB
:1038F0000F0E0C6E01C10BF018EC09F0100E0C6EDF
:1039000002C10BF018EC09F0110E0C6E03C10BF0A4
:1039100018EC09F007840101BFEC1FF057C100F15A
:1039200058C101F107940A0E0C6E00C10BF018EC9F
:1039300009F00B0E0C6E01C10BF018EC09F00C0E27
:103940000C6E02C10BF018EC09F00D0E0C6E03C1E9
:103950000BF018EC09F0F3EF1CF007AAF3EF1CF0E2
:1039600007840101BFEC1FF057C100F158C101F1FC
:103970000794060E0C6E00C10BF018EC09F0070E50
:103980000C6E01C10BF018EC09F0080E0C6E02C1B0
:103990000BF018EC09F0090E0C6E03C10BF018ECDB
:1039A00009F0078462C100F163C101F164C102F151
:1039B00065C103F10794120E0C6E00C10BF018ECF8
:1039C00009F0130E0C6E01C10BF018EC09F0140E87
:1039D0000C6E02C10BF018EC09F0150E0C6E03C151
:1039E0000BF018EC09F00798079A0401805181192F
:1039F0007F0B0DE09EA8FED714EE00F081517F0BE7
:103A0000E126E750812B0F01AD6EF5EF1CF090EF32
:103A10000AF018C100F119C101F11AC102F11BC16C
:103A200003F1000E046F000E056F010E066F000E0D
:103A3000076FF5EC1EF029A134EF1DF02051D8B42A
:103A400034EF1DF018C100F119C101F11AC102F1E2
:103A50001BC103F1000E046F000E056F0A0E066F06
:103A6000000E076FF5EC1EF0120001010451001367
:103A700005510113065102130751031312000101EE
:103A8000186B196B1A6B1B6B12002AC182F40401AC
:103A9000300E822739EC0BF02BC182F40401300E7A
:103AA000822739EC0BF02CC182F40401300E8227FE
:103AB00039EC0BF02DC182F40401300E822739EC71
:103AC0000BF02EC182F40401300E822739EC0BF08A
:103AD0002FC182F40401300E822739EC0BF030C183
:103AE00082F40401300E822739EC0BF031C182F4EC
:103AF0000401300E822739EC0BF032C182F404014C
:103B0000300E822739EC0BF033C182F40401300E01
:103B1000822739EC0BF012002FC182F40401300E21
:103B2000822739EC0BF030C182F40401300E822779
:103B300039EC0BF031C182F40401300E822739ECEC
:103B40000BF032C182F40401300E822739EC0BF005
:103B500033C182F40401300E822739EC0BF01200DD
:103B6000060E1D6E060E1E6E060E1F6E1D2EB6EF85
:103B70001DF01E2EB6EF1DF01F2EB6EF1DF08B842C
:103B8000020E1D6E020E1E6E020E1F6E1D2EC6EF61
:103B90001DF01E2EC6EF1DF01F2EC6EF1DF08B94DC
:103BA00012000101005305E1015303E1025301E159
:103BB000002B94EC1EF0BFEC1FF03951006F3A510E
:103BC000016F420E046F4B0E056F000E066F000E64
:103BD000076FD5EC1EF000C104F101C105F102C16F
:103BE00006F103C107F118C100F119C101F11AC1B1
:103BF00002F11BC103F107B202EF1EF0C9EC1EF087
:103C000004EF1EF0C4EC1EF000C118F101C119F15F
:103C100002C11AF103C11BF11200BFEC1FF059C120
:103C200000F15AC101F1060E2FEC09F0E8CF04F1C2
:103C3000070E2FEC09F0E8CF05F1080E2FEC09F084
:103C4000E8CF06F1090E2FEC09F0E8CF07F1C4EC3C
:103C50001EF000C124F101C125F102C126F103C10A
:103C600027F1290E046F000E056F000E066F000E7F
:103C7000076FD5EC1EF0EE0E046F430E056F000EBD
:103C8000066F000E076FC9EC1EF024C104F125C1B8
:103C900005F126C106F127C107F1D5EC1EF000C1E0
:103CA0001CF101C11DF102C11EF103C11FF1120E71
:103CB0002FEC09F0E8CF04F1130E2FEC09F0E8CF58
:103CC00005F1140E2FEC09F0E8CF06F1150E2FECDC
:103CD00009F0E8CF07F10D0E006F000E016F000E26
:103CE000026F000E036FD5EC1EF0180E046F000E6D
:103CF000056F000E066F000E076FF5EC1EF01CC17D
:103D000004F11DC105F11EC106F11FC107F1C9EC87
:103D10001EF06A0E046F2A0E056F000E066F000E6D
:103D2000076FC4EC1EF01200BF0EFA6E200E3A6F41
:103D3000396BD8900037013702370337D8B0A5EF79
:103D40001EF03A2F9AEF1EF039073A070353D8B402
:103D500012000331070B80093F6F03390F0B010F6E
:103D6000396F80EC5FF0406F390580EC5FF0405DAB
:103D7000405F396B3F33D8B0392739333FA9BAEFA9
:103D80001EF04051392712000101E4EC1FF0D8B0B9
:103D90001200010103510719346FA7EC1FF0D890EE
:103DA0000751031934AF800F12000101346BCBECC3
:103DB0001FF0D8A0E1EC1FF0D8B01200B6EC1FF055
:103DC000BFEC1FF01F0E366FF7EC1FF00B35D8B0AD
:103DD000A7EC1FF0D8A00335D8B01200362FE4EFBF
:103DE0001EF034B1CEEC1FF012000101346B04510F
:103DF0000511061107110008D8A0CBEC1FF0D8A0C0
:103E0000E1EC1FF0D8B01200086B096B0A6B0B6B6A
:103E1000F7EC1FF01F0E366FF7EC1FF007510B5D2C
:103E2000D8A41FEF1FF006510A5DD8A41FEF1FF0A2
:103E30000551095DD8A41FEF1FF00451085DD8A0FB
:103E400032EF1FF00451085F0551D8A0053D095F0E
:103E50000651D8A0063D0A5F0751D8A0073D0B5F69
:103E6000D8900081362F0CEF1FF034B1CEEC1FF04C
:103E7000346BCBEC1FF0D890FBEC1FF007510B5DBF
:103E8000D8A44FEF1FF006510A5DD8A44FEF1FF0E2
:103E90000551095DD8A44FEF1FF00451085DD8A06B
:103EA0005EEF1FF0003F5EEF1FF0013F5EEF1FF07F
:103EB000023F5EEF1FF0032BD8B4120034B1CEECFA
:103EC0001FF012000101346BCBEC1FF0D8B01200D0
:103ED00000EC20F0200E366F003701370237033731
:103EE00011EE33F00A0E376FE7360A0EE75CD8B0F2
:103EF000E76EE552372F74EF1FF0362F6CEF1FF08F
:103F000034B12981D890120001010A0E346F200EBD
:103F1000366F11EE29F03451376F0A0ED890E65201
:103F2000D8B0E726E732372F8FEF1FF00333023385
:103F300001330033362F89EF1FF0E750FF0FD8A071
:103F40000335D8B0120029B1CEEC1FF01200045195
:103F500000270551D8B0053D01270651D8B0063DD0
:103F600002270751D8B0073D032712000051086F00
:103F70000151096F02510A6F03510B6F12000101C9
:103F8000006B016B026B036B12000101046B056B8C
:103F9000066B076B12000335D8A012000351800B8B
:103FA000001F011F021F031F003FDEEF1FF0013F34
:103FB000DEEF1FF0023FDEEF1FF0032B342B032553
:103FC00012000735D8A012000751800B041F051FEF
:103FD000061F071F043FF4EF1FF0053FF4EF1FF02B
:103FE000063FF4EF1FF0072B342B07251200003794
:103FF000013702370337083709370A370B37120002
:104000000101296B2A6B2B6B2C6B2D6B2E6B2F6B8D
:10401000306B316B326B336B120001012A510F0B85
:104020002A6F2B510F0B2B6F2C510F0B2C6F2D5117
:104030000F0B2D6F2E510F0B2E6F2F510F0B2F6F5C
:1040400030510F0B306F31510F0B316F32510F0B5D
:10405000326F33510F0B336F120000011550FF0AFE
:1040600001E11200390EC86E800EC76E280EC66EB2
:10407000000EC56E1450000AD8B468EF20F014503A
:10408000010AD8B481EF20F01450020AD8B49AEF94
:1040900020F01450030AD8B4B3EF20F01450040AEF
:1040A000D8B4DBEF20F01450050AD8B4F4EF20F0B8
:1040B0001450060AD8B40DEF21F01450070AD8B4F2
:1040C00026EF21F01450080AD8B43FEF21F0120077
:1040D0001550000AD8B45EEF21F01550010AD8B48B
:1040E00062EF21F01550020AD8B466EF21F01550A6
:1040F000030AD8B46AEF21F01550040AD8B4D9EFF6
:1041000021F01550000AD8B46EEF21F01550010AC5
:10411000D8B472EF21F01550020AD8B476EF21F02E
:104120001550030AD8B47AEF21F01550040AD8B418
:10413000D9EF21F01550000AD8B47EEF21F01550C8
:10414000010AD8B482EF21F01550020AD8B486EFE4
:1041500021F01550030AD8B48AEF21F01550040A53
:10416000D8B4D9EF21F01550000AD8B497EF21F058
:104170001550010AD8B49BEF21F01550020AD8B4AB
:104180009FEF21F01550030AD8B4B3EF21F015507A
:10419000040AD8B4B7EF21F01550050AD8B4BBEF24
:1041A00021F01550060AD8B4BFEF21F01550070AC8
:1041B000D8B4C2EF21F01550000AD8B4C6EF21F0F0
:1041C0001550010AD8B4CAEF21F01550020AD8B42C
:1041D000CEEF21F01550030AD8B4D2EF21F01550DC
:1041E000040AD8B4D5EF21F01550000AD8B4DDEF99
:1041F00021F01550010AD8B4E1EF21F01550020A60
:10420000D8B4E5EF21F01550030AD8B4E9EF21F056
:104210001550040AD8B4D9EF21F01550000AD8B4CB
:10422000F3EF21F01550010AD8B4F7EF21F0155043
:10423000020AD8B4FBEF21F01550030AD8B4FFEFFF
:1042400021F01550040AD8B4D9EF21F01550000A16
:10425000D8B400EF22F01550010AD8B404EF22F0D0
:104260001550020AD8B408EF22F01550030AD8B44A
:104270000CEF22F01550040AD8B4D9EF21F01550F4
:10428000000AD8B40DEF22F01550010AD8B411EF8E
:1042900022F01550020AD8B415EF22F01550030A87
:1042A000D8B419EF22F01550040AD8B41AEF22F04E
:1042B0001550050AD8B41DEF22F012009E96C58055
:1042C000152A1200E20EC96E152A1200770EC96E69
:1042D000152A1200020EC96E152A12009E96C5807C
:1042E000152A1200E20EC96E152A1200790EC96E47
:1042F000152A1200000EC96E152A12009E96C5805E
:10430000152A1200E20EC96E152A12007A0EC96E25
:10431000152A120017BC03D0DAC1E8FF04D01750E9
:10432000E844E8441F09E8CFC9FF152A12009E9609
:10433000C580152A1200E20EC96E152A120011BAA4
:1043400003D011BC01D003D0050E146E3ED0010184
:10435000D667AFEF21F0100EC96EB1EF21F0D6C1D4
:10436000C9FF152A1200D7C1C9FF152A1200D8C1EA
:10437000C9FF152A1200D9C1C9FF152A1200C58428
:10438000152A1200FF0E156E1C9E12009E96C58007
:10439000152A1200E20EC96E152A1200760EC96E99
:1043A000152A1200C584152A1200FF0E156E1C9ED8
:1043B0001200C584142A156A12009E96C580152A1B
:1043C0001200E20EC96E152A12007B0EC96E152A64
:1043D000120011AA04D0230EC96E152A12001C0E59
:1043E000C96E152A12009E96C580152A1200E20E8B
:1043F000C96E152A12007C0EC96E152A1200E9D763
:104400009E96C580152A1200E20EC96E152A12006A
:104410007D0EC96E152A1200DCD79E96C580152A1E
:104420001200E20EC96E152A12007E0EC96E152A00
:104430001200CFD7C584152A1200FF0E156E1C9EE0
:1044400012001550FF0AD8B4DFEF22F0390EC86E03
:10445000800EC76E280EC66E000EC56E1450000A80
:10446000D8B43AEF22F01450010AD8B44EEF22F03B
:10447000DFEF22F01550000AD8B48CEF22F015506F
:10448000010AD8B490EF22F01550020AD8B49AEF7E
:1044900022F01550030AD8B49DEF22F01550000AFF
:1044A000D8B4A3EF22F01550010AD8B4A7EF22F038
:1044B0001550020AD8B4B1EF22F01550030AD8B44F
:1044C000B4EF22F01550040AD8B4BAEF22F0155018
:1044D000050AD8B4BDEF22F01550060AD8B4C3EFD0
:1044E00022F01550070AD8B4C6EF22F01550080A7A
:1044F000D8B4CCEF22F01550090AD8B4CFEF22F08F
:1045000015500A0AD8B4D5EF22F015500B0AD8B4CA
:10451000D8EF22F0DFEF22F09E96C580DEEF22F08A
:1045200016B004D04E0EC96EDEEF22F0500EC96EEA
:10453000DEEF22F0C584DEEF22F0142AFF0E156EA6
:104540001280DFEF22F09E96C580DEEF22F016B0DB
:1045500004D04F0EC96EDEEF22F0510EC96EDEEFB1
:1045600022F0C586DEEF22F0C9CF23F0C59AC588B8
:10457000DEEF22F0C586DEEF22F0C9CF24F0C59A27
:10458000C588DEEF22F0C586DEEF22F0C9CF25F028
:10459000C59AC588DEEF22F0C586DEEF22F0C9CFCE
:1045A00026F0C58AC588DEEF22F0C584DEEF22F052
:1045B000FF0E156E12861C9CDFEF22F0152A1200EA
:1045C00012B012D012B213D012B414D012A612002C
:1045D00007B01200129623C027F024C028F025C08F
:1045E00029F026C02AF012001290128212001292B4
:1045F0001284120000011550FF0A04E11294156A9A
:0646000021EC22F0120083
:10BF0000E844F926000C160C2B0C3F0C520C640C68
:10BF1000760C860C960CA50CB30CC10CCF0CDC0C6B
:06BF2000E80CF40C000C1B
:00000001FF
